:100000000C942A000C9434000C9434000C943400AA
:100010000C9434000C9434000C9434000C94340090
:100020000C9434000C9434000C9434000C94340080
:100030000C9434000C9434000C9434000C94340070
:100040000C9434000C9434000C9434000C94340060
:100050000C94340011241FBECFE5D8E0DEBFCDBF25
:100060000E9454000C944E010C94000080E487B967
:1000700087E886B9089597B1907E97B997B1877050
:10008000892B87B9369A349BFECF349A24B135B187
:10009000C901089520E040E050E0CA010197F1F75E
:1000A0002F5F2A30D1F70895AF92BF92CF92DF929F
:1000B000EF92FF920F931F93CF93DF930E9418014B
:1000C00080E487B987E886B920E040E050E0CA01C3
:1000D0000197F1F72F5F2A30D1F781E06FEF0E948F
:1000E000220182E06FEF0E94380180E3E82E85E76D
:1000F000F82EAA24BB2487B1807E87B987B187B93F
:10010000369A349BFECF349A04B115B187B1807E04
:1001100087B9389A369A349BFECF349AC4B1D5B198
:1001200087B1807E87B9399A369A349BFECF349A4C
:10013000C4B0D5B081E0C431D80760F4043C1105E7
:1001400080F584ECC816D10408F051C0C5010197B0
:10015000F1F7D1CF81E06FEF0E94220181E06FEFD4
:100160000E9438010A3B110518F4CA50D14090F1A1
:1001700087B1807E87B987B187B9369A349BFECF25
:10018000349A04B115B187B1807E87B9389A369A0E
:10019000349BFECF349AC4B1D5B1C7010197F1F7B2
:1001A000E1CF81E06FEF0E94220181E06FEF0E94BA
:1001B000380187B1807E87B987B187B9369A349B79
:1001C000FECF349A84B195B1F7013197F1F78A3BAC
:1001D000910578F781E06FEF0E94220182E06FEFD6
:1001E0000E94380184ECC816D10408F4AFCF82E035
:1001F0006FEF0E94220182E06FEF0E94380187B109
:10020000807E87B9399A369A349BFECF349A84B16E
:1002100095B1F7013197F1F78A3B910580F781E0BD
:100220006FEF0E94220182E06FEF0E9438018ECFB3
:1002300081EA8FBD83E08EBD8D9A8C9A84B38F60E6
:1002400084BB0895882371F0823079F0813011F4F5
:10025000A998A89A2FB7F894862F90E09BBD8ABDE5
:100260002FBF0895A898A998F5CFA898A99AF2CF7A
:10027000882371F0823079F0813011F4AB98AA9A1A
:100280002FB7F894862F90E099BD88BD2FBF0895B1
:10029000AA98AB98F5CFAA98AB9AF2CFF894FFCF73
:00000001FF
